:10000000012807309F0003108316031300300318E4
:1000100001309F001E3085000310003003180130AE
:10002000860003108312031300300318013086008A
:1000300005100130F0008312031370088607831245
:100040000313851C242825282E280514E830E627CC
:10005000831203130510E830E6271F281430E62723
:06006000312819280028D8
:100FCC00F1000430F2005330F300ED2FED2F01301F
:100FDC00F302031DF22FF32FEC2F0130F202031D4D
:100FEC00F82FF92FE92F0130F102031DFE2FFF2FEF
:040FFC00E72F0800D3
:02400E00693F08
:00000001FF
